:020000020000FC
:1000000045C063BFC3C7CBCFD3D7DADEE1E5E8EBAA
:10001000EEF0F3F5F7F9FAFCFDFEFEFEFEFEFEFD46
:10002000FCFBFAF8F6F4F2EFECE9E6E3E0DCD8D515
:10003000D1CDC9C5C1BDB9B5B1ADA9A6A29E9B9888
:1000400095928F8C8A88868483828180808080804C
:10005000808182848587898B8E909396999DA0A4B8
:10006000A7ABAFB3B7BB1205FA05FA05FA05FA0557
:10007000FA05FA0AFA0AFA0AFA14FA14FA14FA0F42
:10008000FA1EC828642364236419C8000FE50DBF55
:1000900000E810E006BD16BD0AE213E3177F026018
:1000A0000160006800640F7D0F7E1B7F1D7F116063
:1000B0000ABD13BFB89A3CE352E3E6E6F0E0C89508
:1000C000702D3196CF0173957A95B9F3FC01C895DF
:1000D000302D0196FC01C895502D019653955A95E7
:1000E00099F3E2E0F0E0C895202D3196C89509BC5F
:0C00F000432F4A95F1F72A95C1F7F1CF94
:00000001FF
